:1000000083177D3084007E30072083010F28640031
:100010008001840A0406031900340406082800300D
:10002000A2000030A3000030A0000030A1000310A7
:1000300083160313003003180130850003100030CD
:10004000031801308600A426F32783120313200827
:10005000013EA00021080318013E003EA10000302F
:10006000A2000030A300342820082207013E0927FF
:10007000B8002208243E8313840038088000013031
:10008000A2070318A30A0030A3072308803AB80088
:1000900080303802031D4E2810302202031C5128E4
:1000A000522834280310003003180130B900003002
:1000B0007226003083120313A2000030A3006028D0
:1000C0002208243E831384000008EE2583120313C4
:1000D0000130A2070318A30A0030A3072308803ABF
:1000E000B80080303802031D772808302202031C34
:1000F0007A287B2860280310003003180130B900EB
:1001000001307226083083120313A2000030A300CE
:1001100089282208243E831384000008EE258312D8
:1001200003130130A2070318A30A0030A307230812
:10013000803AB80080303802031DA0281030220217
:10014000031CA328A4288928C830D72783120313A7
:100150002008103E013E09270038031DB028B128B1
:0E016000B5280030A0000030A100252800289E
:100BDC00B9003908860019260D3083120313BA00A8
:100BEC00F82DF82D0130BA02031DFD2DFE2DF72D29
:100BFC000800BE000310003003180130BF003E1C7B
:100C0C00082E092E0D2E3D08C0004008BF0703100A
:100C1C00BD0D0310BE0CBE08031D152E162E052E81
:100C2C003F08182E0800FD147D0885001130BB000C
:100C3C00202E202E0130BB02031D252E262E1F2E0A
:100C4C007D157D0885001130BC002D2E2D2E013018
:100C5C00BC02031D322E332E2C2EFB30BE003E0860
:100C6C00FD057D0885001130BD003D2E3D2E013067
:100C7C00BD02031D422E432E3C2E0800FD30C10048
:100C8C004108FD057D0885001130BE004E2E4E2E0C
:100C9C000130BE02031D532E542E4D2E7D157D08A2
:100CAC0085001130BF005B2E5B2E0130BF02031D8F
:100CBC00602E612E5A2EFB30C1004108FD057D08C7
:100CCC0085001130C0006B2E6B2E0130C002031D4D
:100CDC00702E712E6A2E0800BA000230860044264F
:100CEC000A30D727283083120313BD003A08FF259A
:100CFC0083120313BC0039083C07BA000310003000
:100D0C0003180130B9009D2E143086004426213082
:100D1C0083120313BB00932E932E0130BB02031DD1
:100D2C00982E992E922E0130BC003C08B9073A0837
:100D3C003902031CA22EA32E8A2E080038308312EF
:100D4C000313860044260530D7273830831203134B
:100D5C0086004426213083120313B900B62EB62E1A
:100D6C000130B902031DBB2EBC2EB52E38308600C7
:100D7C004426213083120313BA00C52EC52E013030
:100D8C00BA02031DCA2ECB2EC42E38308600442640
:100D9C00213083120313BB00D42ED42E0130BB029E
:100DAC00031DD92EDA2ED32E013086004426323084
:100DBC00D7270D308312031386004426213083126B
:100DCC000313BC00EA2EEA2E0130BC02031DEF2EE9
:100DDC00F02EE92E063086004426213083120313B0
:100DEC00BD00F92EF92E0130BD02031DFE2EFF2E83
:100DFC00F82E0800FE00FE1F082F83137E188317A1
:100E0C00000808000408FE0007308A007E088207EC
:100E1C0000342E342E342E34503452344F34473464
:100E2C00523441344D3441342034503441345234F2
:100E3C0041342034453453344334523449344234ED
:100E4C0049345234203455344E3420344D344534E6
:100E5C004E34533441344A344534203445344E34C2
:100E6C00203455344E3420344434493453345034C3
:100E7C004C344134593420344C34433444342034CD
:100E8C003134363420345834203431342C3420343A
:100E9C0043344F344E3420345334433452344F346F
:100EAC004C344C3449344E34473420344334493474
:100EBC005234433455344C34413452342E342E3461
:100ECC002E34503452344F344734523441344D3430
:100EDC0041342034503441345234413400340034E1
:100EEC000034003400340034003400340034003456
:100EFC000034003400340034003400340034003446
:100F0C000034003400340034003400340034003435
:100F1C000034003400340034003400340034003425
:100F2C000034003400340034003400340034003415
:100F3C000034003400340034003400340034003405
:100F4C0000340034003400340034003400340034F5
:100F5C0000340034003400340034003400340034E5
:100F6C0000340034003400340034003400340034D5
:100F7C0000340034003400340034003400340034C5
:100F8C0000340034003400340034003400340034B5
:100F9C0000340034003400340034003400340034A5
:100FAC00003483120313BE000430BF005330C00062
:100FBC00E02FE02F0130C002031DE52FE62FDF2FBD
:100FCC000130BF02031DEB2FEC2FDC2F0130BE02D2
:100FDC00031DF12FF22FDA2F0800013083120313B7
:0A0FEC00860044260A30D7270800CB
:02400E00693F08
:00000001FF
